:020000040000FA
:10000000AC28040000000000B2230000B22300006E
:10001000B2230000B2230000B2230000B22300008C
:10002000B2230000B2230000B2230000B22300007C
:10003000B2230000CE230000B2230000B223000050
:10004000B2230000B2230000B22300003E260000CD
:10005000B2230000B2230000B2230000B22300004C
:10006000B2230000B2230000B2230000B22300003C
:10007000B2230000B2230000B2230000B22300002C
:10008000B2230000B2230000B2230000B22300001C
:10009000B2230000B2230000B2230000B22300000C
:1000A000B2230000B2230000B2230000B2230000FC
:1000B000B2230000B2230000B2230000B2230000EC
:1000C000B2230000B2230000B2230000B2230000DC
:1000D000B2230000B2230000B2230000B2230000CC
:1000E000B2230000B2230000B2230000B2230000BC
:1000F000B2230000B2230000B2230000B2230000AC
:10010000B2230000B2230000B2230000B22300009B
:10011000B2230000B2230000B2230000B22300008B
:10012000B2230000B2230000B2230000B22300007B
:10013000B2230000B2230000B2230000B22300006B
:10014000B2230000B2230000B2230000B22300005B
:10015000B2230000B2230000B2230000B22300004B
:10016000B2230000B2230000B2230000B22300003B
:10017000B2230000B2230000B2230000B22300002B
:10018000B2230000B2230000B2230000B22300001B
:10019000B2230000B2230000B2230000B22300000B
:1001A000B2230000B2230000B2230000B2230000FB
:1001B000B2230000B2230000B2230000B2230000EB
:1001C000B2230000B2230000B2230000B2230000DB
:1001D000B2230000B2230000B2230000B2230000CB
:1001E000B2230000B2230000B2230000B2230000BB
:1001F000B2230000B2230000B2230000B2230000AB
:10020000A4280000000000008344550050000000B6
:1002100000277800000006000A0000008444520015
:100220004F5000003E007800000006000A00000069
:1002300084535700414200000080FD00000006008A
:100240000A000000834E4900500000000E87E800BD
:10025000000006000A000000C4545500434B000093
:100260001E27780010079800000006000C00000010
:10027000C4535700415000009E1F7800000F7800C3
:100280004F007800000006000E000000C44F56002A
:1002900045520000002778001E0090000000060074
:1002A0000C000000C3524F0054000000801F780073
:1002B0001E0090003E0F78004F27780000000600D7
:1002C00010000000C4504900434B00000000E9004A
:1002D000000040006E007800000006000E000000E4
:1002E000C4504F004B4500000000E90000004000F2
:1002F0000E0040003E0878003E0078000000060036
:1003000012000000C4524F004C4C00000000E900F5
:100310000C003400811F7800821F78008E0040009E
:1003200081004000911F7800010178000000E90081
:1003300000800900C21078004F0F78004F0178004C
:10034000CF0078003E007800000006002600000084
:10035000C43F4400555000000000B00001003200CE
:1003600000277800000006000E000000823E5200C8
:10037000801F78003E007800000006000A000000A0
:1003800082523E00002778004F00780000000600EF
:100390000A00000082524000002778007FB89700D2
:1003A000000006000A0000008140000010007800F4
:1003B0000000060008000000C24340001040780022
:1003C0000000FB00000006000A000000C121000040
:1003D0003E0878003E007800000006000A00000099
:1003E000C24321001E4878003E0078003E0078009D
:1003F000000006000C000000812B00003E004000C1
:100400000000060008000000C22B2B00811F7800AE
:10041000BE0078003E0040001E8F4800CF007800EC
:100420000000060010000000864E450047415400C1
:10043000450000000000EA00000006000C0000007B
:10044000812D00003E0010000000060008000000A2
:10045000C22D2D00811F7800BE0078003E001000E4
:100460001E8F1800CF00780000000600100000006A
:1004700082322A004100DD00000006000800000072
:1004800082342A004200DD0000000600080000005F
:1004900082322F004180DE000000060008000000CC
:1004A00082342F004280DE000000060008000000B9
:1004B00082303C004F80DE00000006000800000093
:1004C000C2303D000000B000010032000080EF00AB
:1004D0000080EA00000006000E000000C2303E006E
:1004E0000000B000020032000080EA004F80DE0011
:1004F000000006000E000000C2553C003E00100047
:100500000000EF00F2FF3900000006000C000000C0
:10051000C13C00003E0010000000EF00ECFF350081
:10052000000006000C000000C13D00003E00680015
:100530000000EF00E6FF3200000006000C000000A3
:10054000C13E00003E0010000000EF00E0FF3C0054
:10055000000006000C000000C34E4F0054000000D5
:100560000000B000DAFF32000000EF0000000600DB
:100570000E000000C2552A00811F78003E00B8001E
:10058000CF007800000006000C000000C12A000027
:10059000811F78003E80B900CF007800000006007F
:1005A0000C000000C5552F004D4F4400821F7800FD
:1005B000811F7800000178001E00780011000900FA
:1005C0000280D800010F7800CF0078004F0178003A
:1005D000000006001A000000C6552A002F4D4F00EB
:1005E00044000000821F7800811F7800000178001D
:1005F0003E0078001E00B800110009004288D800B3
:10060000010F7800CF0078004F017800000006004D
:100610001E000000C52A2F004D4F4400821F7800A5
:10062000811F7800000178003E0078001E80B9002C
:10063000110009004208D800010F7800CF007800AF
:100640004F017800000006001C000000C42F4D0080
:100650004F440000821F7800811F7800000178005D
:100660001E007800110009000200D800010F780078
:10067000CF0078004F017800000006001A0000004B
:10068000C12F0000811F780080007800F1FF070073
:1006900001F0A300010039008100EA00801F78000A
:1006A0003E00780000F0A300010039000000EA00DD
:1006B0004100DD00810050004F007800CF0078003D
:1006C0000500390000F0A300020031000000E8003E
:1006D000000006000000E9000000060030000000F5
:1006E000C34D4F0044000000DAFF07003E007800D1
:1006F000000006000C000000C22A2F00811F7800B5
:1007000080007800C5FF0700E1FF37000000060009
:100710000E000000C453510052540000831F7800A3
:10072000821F7800811F78000027EB00010820005D
:100730001E8140000211B8000200E10001003900F2
:100740001E8F40008100D100F9FF39001E01E80032
:100750001E11B8000010E100010031001E0FE8007A
:10076000CF0078004F017800CF0178003E0078007C
:100770000000060032000000C34D41005800000098
:100780001E00E10002003C003E0078000000060070
:10079000620747000000060012000000C34D490038
:1007A0004E0000001E00E100F9FF35003E00780019
:1007B000000006000E000000C3414200530000008C
:1007C0000000B00001003B000000EA00000006004D
:1007D0000E00000083414E00440000003E00600017
:1007E000000006000A000000824F52003E00700028
:1007F000000006000800000083584F00520000006F
:100800003E006800000006000A000000C3415300DB
:10081000480000000000B0000800320004003B0067
:100820000080EA00008009001E8FD100030037001D
:100830000000E900008009001E0FD0003E00780093
:10084000000006001E000000C34C530048000000DA
:100850000000B000F9FF3200F5FF3B000080EA0025
:10086000008009001E0FD100F4FF370000000600D1
:1008700016000000C3524F004C0000000000B00002
:10088000EEFF320004003B000080EA000080090017
:100890001E0FD300E9FF37000000E90000800900C7
:1008A0001E0FD200E5FF3700000006001E0000000A
:1008B00083434F004D0000000080EA000000060066
:1008C0000A000000C32B430021000000811F7800B4
:1008D000BE00780010C840003E007800CF007800CD
:1008E0000000060012000000C32D4300210000009C
:1008F000811F7800BE00780010C810003E0078000C
:10090000CF0078000000060012000000C22B21007A
:10091000811F7800BE007800108840003E007800FB
:10092000CF0078000000060010000000C22D21005A
:10093000811F7800BE007800108810003E0078000B
:10094000CF0078000000060010000000C4464900F7
:100950004C4C0000821F7800811F78003E01780017
:10096000BE0078000201E90002800900805878008A
:100970003E007800CF0078004F01780000000600AC
:100980001C000000C5434D004F564500821F7800F3
:10099000811F78003E0178009E001100BE007800A3
:1009A000050039000000E90009003300008009005B
:1009B00031597800060037000201400081004000F4
:1009C0000000E90002003300008009004161780066
:1009D0003E007800CF0078004F017800000006004C
:1009E00030000000C44D4F0056450000821F7800C3
:1009F000811F78003E0178009E001100BE00780043
:100A0000050039000000E9000B00330000800900F8
:100A1000311978000800370002014000020140004F
:100A200081004000810040000000E9000200330026
:100A300000800900412178003E007800CF00780056
:100A40004F01780000000600340000008449440093
:100A50004C4500000140FE00000006000A000000B6
:100A600085534C00454550000040FE000000060044
:100A70000A000000C8535F0054414D00504F4E0023
:100A80000027780000902000000006000E00000003
:100A9000C6535F00574F5200440000000027780003
:100AA00000962000000006000E000000C8535F0002
:100AB000464F52004D41540000277800009A200014
:100AC000000006000E000000C549540052583100D5
:100AD0000027780000A02000000006000C000000A5
:100AE000C55445004C4543000027780040A0200035
:100AF000000006000C000000C6434E00544954009C
:100B0000500000000027780060A0200000000600D0
:100B10000E000000C8534500515545004E434500A6
:100B20000027780080A02000000006000E000000D2
:100B3000C3504100440000000027780020A120009D
:100B4000000006000C000000C33E49004E000000FB
:100B50000027780040A12000000006000C000000E3
:100B6000C94D45004D5F4400455054004800000009
:100B70000027780060A1200000000600100000009F
:100B8000CB4D45004D5F500052474800455245004F
:100B90000027780080A1200000000600100000005F
:100BA000CA414400525F4300524541005445000091
:100BB00000277800C0A120000000060010000000FF
:100BC000C5535400415254000027780000A2200071
:100BD000000006000C000000C55445004D505300B5
:100BE0000027780040A22000000006000C00000052
:100BF000C84D45004D5F480045524500002778002C
:100C000080A22000000006000E000000CA5354001D
:100C10004F505F00464F52005448000000277800B4
:100C2000A0A220000000060010000000C4454F00F4
:100C30004C4E000000277800E0A2200000000600D3
:100C40000C000000C3454F0046000000002778005C
:100C500000A32000000006000C000000C442410078
:100C6000534500000027780020A320000000060064
:100C70000C000000C5535400415445000027780083
:100C800040A32000000006000C000000C5455200F3
:100C9000524F52000027780060A320000000060099
:100CA0000C000000C5495400314D53000027780066
:100CB000C0A32000000006000C000000CA494E003E
:100CC000505554005F4649004C450000002778000D
:100CD00000A420000000060010000000C7505200D1
:100CE000475F50004E5400000027780040AF2000BE
:100CF000000006000E000000C544450050544800A6
:100D000000277800E08F20000E0050004180DE00B8
:100D10000000060010000000C65244004550540078
:100D20004800000000277800408020000080570025
:100D30004180DE000000060012000000C750520093
:100D4000474845005245000091FF07000027780002
:100D5000801F78003E0078002000B000100078006E
:100D6000002778004F00780010007800000006008F
:100D70001C000000C83E5000524748004552450044
:100D800083FF070000277800801F78003E0078006E
:100D90008FFD0700002778004F0078002000B0008A
:100DA0008BFD0700000006001C000000C4454D003C
:100DB0004954000000277800002778003001200007
:100DC000DAFD070033FD070000277800100120003E
:100DD000D6FD07003E007000E1FD07000000B000F6
:100DE0003E0078001E0032003FFF07001000780030
:100DF0000000B0003E0078000E00320000277800AE
:100E000080BB200038FF070071FD07000027780035
:100E1000A0002000C5FD07000000B0003E007800E3
:100E20000300320000277800E002200001003700B4
:100E300000000600002778000000B0003E007800A7
:100E400007003200A1FF07002008B0005BFD07008B
:100E50009CFD07000000B0003E007800F9FF320062
:100E600000277800E020200010007800002778009C
:100E7000002020003E0060000000B0003E0078002E
:100E80000300320000277800000020000500370032
:100E900000277800002120004DFD07000027780082
:100EA000F0FF2F000000B0003E007800ECFF3200A1
:100EB0000000060086000000C450520047400000B9
:100EC00089FF0700811F7800821F7800BE0078002C
:100ED0001000A7001500370002FC2F0002816000FF
:100EE0001010E10011003A00100190001E10E10006
:100EF0000E003A004000B000E103B2000080400064
:100F0000C108DE00008040000001EB000000A600E8
:100F1000B0007800304178000000A600B0007800F2
:100F2000020F78000100780005003700220320003E
:100F30001E0978001181BA00020F78001100BA0072
:100F40004F017800CF007800000006004C00000040
:100F5000C45052004721000063FF0700811F780042
:100F6000821F7800BE00780002FC2F000281600022
:100F70001010E10003003A00100190001E10E10083
:100F8000060032001000A6002800070002FC2F0017
:100F9000029860001E107800110007004000B000A9
:100FA000E103B20000804000C108DE000080400084
:100FB00062074700BE0078003E0178000000A600EE
:100FC00001187800025878000000A6000118780087
:100FD0003E0078004F017800CF0078000000060046
:100FE000811F7800821F7800831F7800841F78009B
:100FF000B00078002203200030097800F3002000C0
:101000001101BA003182BA00021878000458780041
:101010001101BA003182BA00045878000218780031
:101020008301E900F6FF31002C003700811F7800B2
:10103000821F7800831F7800841F7800210420001D
:10104000020E2000911F780091087100B000780016
:10105000227620000119780010097800120424007B
:10106000023B880052052000323B8800A20A200083
:10107000323B880061E7A80000000000000000008B
:1010800012002400023B880022032000300978006F
:10109000F300200030017800304278008208BB0065
:1010A0008498BB0030427800300178008208BB0091
:1010B0008498BB008301E900F6FF3100520520004F
:1010C000323B8800A20A2000323B880061E7A8007A
:1010D00000000000000000004200F9004006B100DE
:1010E0004F027800CF0178004F017800CF007800E0
:1010F00000000600D4000000C4505200472C00003D
:1011000011FF070063FC070062FC0700002778005E
:10111000000020000027780020002000BBFC070012
:1011200017FF07008CFF0700000006001C000000EE
:10113000C445450050400000811F78002103200075
:10114000BE0878001000BA00CF007800000006004A
:1011500012000000C445450050210000811F7800A6
:1011600062A7B7009E007800213B8800410424005C
:10117000013B88000500FC0051052000313B880040
:10118000A10A2000313B880061E7A80000000000B0
:101190000000000061E7AF00FEFF370021032000E0
:1011A000BE0878003E08BB0041002400013B8800D7
:1011B0000500FC0051052000313B8800A10A2000F9
:1011C000313B880061E7A80000000000000000003B
:1011D00061E7AF00FEFF37003E007800CF007800E7
:1011E000000006004A000000CB7370005F737900B6
:1011F0006E63700072672100BBFE07001000A6003E
:101200008AFF07001000A0003E00780000000600E2
:1012100060000000C44845005245000077FE07000A
:1012200010007800000006000C000000C53E4800D9
:101230004552450071FE070065FC070000000600EE
:101240000C000000C2432C00F4FF070000277800C8
:101250001000B000F7FF070062FC07000000060066
:1012600010000000C12C0000ECFF070000277800F0
:101270002000B000EFFF070055FC0700000006004B
:1012800010000000CA7370005F636F006D7069002A
:101290006C650000FFFB0700FEFB070008FF07006E
:1012A000801F78003E007800002778003E0068002C
:1012B000002778007FB8970000277800F00320000F
:1012C0003E0060001000B0000027780030002000D1
:1012D000E0FC0700E8FB070081FC07003E0010006F
:1012E0004100DD0049FC0700002778004F0078002E
:1012F00000277800000420003E0060000000B000DD
:101300003E007800310032008FFE07000027780091
:101310000000200000277800200020003BFC070090
:101320004CFC0700DBFB070000277800F0FF2F00D4
:101330007EFC07000000B0003E0078000D00320087
:10134000801F78003E0078003E007800002778007B
:1013500070002000002778004F0078004180DE00F8
:1013600000277800000028003E00700064FF07009E
:101370001500370074FE07000027780000002000E9
:10138000002778002000200020FC07001FFC070039
:10139000801F78003E0078000027780020002000A1
:1013A000002778004F00780055FF0700801F780065
:1013B0003E00780000277800000020000027780019
:1013C0004F0078004EFF070017003700B1FB070001
:1013D000B0FB0700BAFE070049FF070000277800AE
:1013E00000002000002778002000200007FC0700F4
:1013F000A8FB0700A7FB0700B1FE070031FC0700B0
:101400009DFB0700002778006000200047FC0700D4
:101410003E0060000000B0003E007800EBFF3200AC
:101420003E0078003E00780000000600E600000064
:101430004249460000277800000B20000027780072
:10144000000020002EFF0700002778008007200002
:1014500000277800E003200029FF0700002778001C
:101460002003200000277800F0FF2F0024FF070052
:1014700035FE07000000060026000000C77370005C
:101480005F73610075740000801F78003E00780073
:10149000801F78003E0078007EFB07007DFB070080
:1014A000002778000000200000277800200020009E
:1014B000E8FB070082FE07003E0078000027780066
:1014C0004F007800002778004F0078000027780050
:1014D000500020007DFB070000277800500020000E
:1014E0007AFB0700DBFB0700801F78003E007800D6
:1014F00000277800F0002000D5FC070000277800C6
:101500004F00780000277800F0FF2F00D0FC070084
:101510003E00400000277800400020007BFB0700D1
:10152000002778004000200078FB070000277800A3
:10153000000020000027780020002000C5FB0700E5
:1015400085FE0700000006008E00000044454C00A8
:101550005345000000277800700320000027780022
:10156000F0FF2F00E6FE0700F7FD0700C6FF0700AB
:10157000F5FD070000000600180000004454480074
:10158000454E0000F0FD0700BFFF07000000060009
:101590000C00000044434100534500000027780040
:1015A00000002000002778000027780000002000BD
:1015B00000277800601B200036FF070000000600AF
:1015C00018000000424F460000277800000020006D
:1015D00000277800A01C20002EFF070000277800BD
:1015E00000002000002778004029200029FF070084
:1015F00090FF0700000006001C00000045454E005B
:10160000444F4600D3FF0700000006000A00000018
:1016100047454E004443410053450000B8FD0700D4
:101620004180DE004CFB07000000B0003E00780067
:1016300025003200002778003000200023FB07003F
:10164000002778003000200020FB07003E007000DB
:101650000000B0003E00780008003200801F7800D3
:101660003E007800B8FD070087FF070000277800DC
:101670004F0078001000B100020037003E007800F3
:101680003E007800002778008EFB07000000B000C5
:101690003E007800E7FF32003E0078000027780027
:1016A0000000200000277800001C2000F9FE070041
:1016B000002778000000200000277800E0102000BC
:1016C000F4FE07000200370000277800F0FF2F002B
:1016D00000000600640000004542450047494E00F6
:1016E00099FD0700000006000A00000045554E0065
:1016F00054494C004FFF07000027780040002000AD
:1017000002FB07000027780040002000FFFA0700D6
:101710005DFF070000000600180000004557480064
:10172000494C450043FF0700000006000A00000086
:1017300046524500504541005400000085FF070017
:101740000027780040002000F0FA0700002778000A
:1017500040002000EDFA07004BFF070000000600E4
:101760001A00000042444F000027780000002000CB
:101770000027780080132000C6FE070072FD0700D6
:10178000002778000000200000277800601B200060
:10179000C0FE070000277800000020000027780026
:1017A000601B2000BBFE07000000060026000000B2
:1017B000452B4C004F4F50000027780000002000C0
:1017C00000277800001C2000B2FE070000277800E8
:1017D0000000200000277800C01F2000ADFE070099
:1017E000002778000000200000277800001C20005F
:1017F000A8FE0700002778000000200000277800DE
:1018000060142000A3FE07000027780000002000DD
:1018100000277800601420009EFE07000027780053
:1018200000002000002778008028200099FE070093
:10183000002778000000200000277800C02A200040
:1018400094FE0700ABFF070000277800000020008F
:1018500000277800E01020008EFE070000277800A7
:101860000000200000277800E010200089FE07001B
:101870000000060064000000C74C490054455200B7
:10188000414C0000002778008007200000277800E6
:10189000007022001AFE070000277800801F7800E1
:1018A0003E0078000027780040FF2F00E8FB07008B
:1018B0000002B000002778004F0078000027780071
:1018C00040002000E2FB07000DFE07004AFE070073
:1018D0000000060030000000444C4F004F50000054
:1018E0000027780010002000E6FF0700B2FF070085
:1018F0000000060010000000814900000027780069
:101900007FB89700000006000A000000814A00002E
:10191000002778005FB89700000006000A0000006A
:10192000814B0000002778003FB8970000000600B8
:101930000A000000854C450041564500002778000C
:101940004F0078004F007800801F7800801F7800DB
:101950003E00780000000600140000008445580096
:10196000495400000000060008000000C243520075
:1019700000277800D00020000EFD07000027780027
:10198000A00020000BFD0700000006001200000070
:10199000C44245004C4C0000002778007000200035
:1019A00004FD0700000006000E000000C5535000B3
:1019B000414345000027780000022000FDFC07009D
:1019C000000006000E000000C653500041434500D1
:1019D0005300000060FA07000000B0003E007800ED
:1019E00008003200F3FF07001000B1000027780064
:1019F000B4FA07000000B0003E007800F9FF3200A2
:101A00003E0078000000060022000000C454590087
:101A10005045000000277800B1FA07000000B00030
:101A20003E0078002F0032001000B100801F7800C7
:101A30003E0078000027780060FA07000027780051
:101A4000F00F20003E006000002778009DFA07009C
:101A500010FA07000027780030002000B3FA0700D2
:101A60003E0070000000B0003E0078000900320027
:101A70003E007800002778004F0078003E00780094
:101A80000027780000002000801F78003E007800CA
:101A90000B0037000027780000277800D0002000D6
:101AA000A2FA07000000B0003E00780003003200F8
:101AB0003E007800AEFF070001003700BDFC0700C4
:101AC0001000B000002778004F0078000027780051
:101AD0007CFA07000000B0003E007800D2FF320020
:101AE00069003700002778004F80DE000000B0005A
:101AF0003E00780064003200801F78003E007800CD
:101B0000E4F90700E3F90700EDFC0700002778007F
:101B10004F0078000000EA00002778000000B000C5
:101B20003E00780014003200801F78003E007800EC
:101B30000027780080FF2F0045FB07000027780072
:101B400000277800D000200078FA07000000B000DD
:101B50003E007800030032003E00780084FF07005A
:101B60000100370093FC0700002778004F00780041
:101B70001000B10002003700BFF907003E007800F6
:101B800000277800801F78003E0078000000B00039
:101B90003E0078001100320000277800002778000E
:101BA000D000200061FA07000000B0003E0078007D
:101BB000030032003E0078006DFF0700010037008F
:101BC0007CFC0700002778004F0078001000B1006F
:101BD000801F78003E007800010037003E0078004A
:101BE0000027780000002000002778002000200057
:101BF00006FA0700A7F90700A6F90700B0FC0700DE
:101C0000002778004F007800002778000000B0001F
:101C10003E00780014003200801F78003E007800FB
:101C20000027780000277800F00F20003E006000B9
:101C30000027780000277800D00020003BFA07003A
:101C40000000B0003E007800030032003E00780043
:101C500047FF07000100370056FC07000027780007
:101C60004F0078001000B1000027780015FA070037
:101C70000000B0003E007800A7FF32003E00780070
:101C80003E0078003E0078003E0078003E0078007C
:101C90000000060046010000C5434F00554E5400A9
:101CA000002778001000B00073F90700C3F907009F
:101CB00000277800F00F20003E00600000000600C2
:101CC00016000000C92D5400524149004C494E00F5
:101CD000470000000027780001FA0700002778007D
:101CE0003000200079F9070000277800300020003C
:101CF00076F907001000B1003E004000AFF9070080
:101D0000002778000002200008FA07003E0060006B
:101D10000000B0003E007800020032001000B10068
:101D2000ECFF37000000060034000000C342490009
:101D30004E0000000027780020002000C9FB0700AB
:101D4000A3F907000000060010000000C54F430083
:101D500054414C000027780080002000C1FB0700A0
:101D60009BF907000000060010000000C744450072
:101D700043494D00414C000000277800A00020009E
:101D8000B8FB070092F907000000060012000000EF
:101D9000C3484500580000000027780000012000DB
:101DA000B0FB07008AF907000000060010000000E1
:101DB000C7434F004E564500525400001000B0007B
:101DC000002778000000200032F907007BF90700A7
:101DD0000027780000277800B0022000D3F9070020
:101DE0000000B0003E007800070032003E0078009E
:101DF000801F78003E0078001000B00000277800B7
:101E00004F0078000C00370000277800D002200037
:101E1000C6F907000000B0003E007800060032005E
:101E2000801F78003E0078001000B0000027780086
:101E30004F0078001000B100801F78003E0078004D
:101E4000002778005DF907000003B1000027780043
:101E50004F80DE000000B0003E0078000400320039
:101E60003E00780000277800F0FF2F003500370093
:101E7000002778000027780090002000B1F90700C3
:101E80000000B0003E007800060032007000B10093
:101E90000027780000277800A00020009DF90700A7
:101EA0000200370000277800000020000000B0008A
:101EB0003E007800040032003E00780000277800E1
:101EC000F0FF2F001F0037000027780065FB070098
:101ED000100078008FF907000000B0003E00780085
:101EE00015003200801F78003E007800801F7800C7
:101EF0003E0078005BFB0700100078009EF90700A9
:101F0000002778004F0078001000B000002778000C
:101F10004F007800D8F80700801F78003E00780056
:101F20003E004000002778004F007800002778002E
:101F300000002000030037003E00780000277800F2
:101F4000F0FF2F000000B0003E007800BCFF320020
:101F5000002778004F0078000000B0003E007800B5
:101F600005003200801F78003E0078000000EA0083
:101F7000002778004F00780000000600E80000000D
:101F8000C23C23000027780000002000CAFA0700A6
:101F900014F9070000277800801F78003E007800C1
:101FA0004F80DE00002778004F00780004FA070019
:101FB000000006001C000000C4484F004C44000014
:101FC000BDFA0700002778001000B0000027780055
:101FD0001000B0000027780030002000BBF8070098
:101FE000F6F8070000277800F00F20003E006000A0
:101FF00000277800E0052000EAF9070063FA0700EF
:1020000000277800EDF8070000277800F00F200087
:102010003E0060001000B00000277800E0052000BE
:10202000E0F907009BF80700EEF807001000B00089
:10203000ECF807000000060042000000C123000089
:1020400008FB07001000780058F907008AF807001D
:102050000003B000002778000027780090032000DC
:1020600038F9070000277800700020003E0060006B
:102070003E004000D2FF07000000060022000000E2
:10208000C2235300EEFF07000027780034F9070051
:102090000000B0003E007800FAFF320000000600A9
:1020A00012000000C4534900474E000079F80700B1
:1020B0000000B0003E0078000300320000277800E6
:1020C000D0022000BEFF070000000600160000003E
:1020D000C2233E003E0078003E00780076FA0700FA
:1020E000EFFE0700000006000E000000C12E0000F9
:1020F000A4FF07000027780000022000B0FF0700BF
:10210000E0FF0700E9FF0700F2FF070041FE0700BC
:102110000000060016000000C13F0000100078001B
:10212000F3FF0700000006000A000000C2552E0061
:10213000002778000000200092FF070000277800A9
:10214000000220009EFF07003E0078004AF80700CA
:10215000CCFF0700DFFF07002EFE0700000006008F
:102160001C000000C4574F0052440000801F78003C
:102170003E00780049FA07000027780000002000A0
:1021800044F8070097F807000027780000002000B7
:10219000A8FA07008EF8070000277800000020004A
:1021A000AAFA07008AF8070063FA0700100078000F
:1021B00067FA0700100078003E0040000027780012
:1021C000801F78003E0078001000B00000277800E3
:1021D000100020005EFA0700CDF907000027780004
:1021E0004F00780075F8070000277800F00F2000F6
:1021F0003E00600000277800801F78003E007800D5
:10220000002778003000200030F807000027780011
:102210006AF807003E0040001000B00071F80700A7
:10222000002778004F00780000277800A5F8070005
:1022300018F807000027780030002000BBF80700DE
:102240003E0070000000B0003E0078000A0032003E
:102250003E00780000277800F0FF2F00002778006C
:1022600074FA07005AF807000027780077FA070089
:1022700057F807002E003700002778000027780065
:10228000D0002000A9F807000000B0003E00780050
:10229000070032003E00780000277800F0FF2F0092
:1022A0000027780063FA070049F80700200037008C
:1022B00000277800801F78003E0078000027780013
:1022C0009000200099F80700002778007FB8970059
:1022D000002778000002200094F807003E007000FC
:1022E000002778004F007800002778007FB897001B
:1022F0008EF807003E0070000000B0003E0078003D
:102300000300320000277800F0FF2F00080037009C
:1023100000277800100020000027780030002000FF
:10232000EAF7070069F9070000277800000020009D
:102330000000B0003E007800A0FF32003E007800B0
:10234000002778004F0078003E007800000006006B
:10235000F8000000C12700000027780000022000DC
:1023600082FF07000027780014F807000000B00083
:102370003E007800CE003200801F78003E007800DA
:1023800011FA070000277800801F78003E007800CF
:102390002000B00010007800002778004F0078007F
:1023A00010007800002778007FB897000027780099
:1023B0000027780001F807003E0040001000B00040
:1023C0000027780040002000C0F7070000277800B1
:1023D00040002000BDF70700AEF70700ADF707008B
:1023E000B7FA070000277800F0F32F003E006000E6
:1023F000002778004F007800A6F707000027780034
:10240000F00F20003E006000A2F70700EBF7070086
:1024100000277800F00F20003E00600043F807001E
:102420000000B0003E007800350032001000B0001F
:102430000027780060002000A4F7070095F7070048
:1024400040F807000000B0003E007800290032008C
:1024500090F707000027780080FF2F00FCF80700A6
:102460008CF70700D5F7070030F807000000B00030
:102470003E0078001C0032001000B00000277800F9
:102480006000200091F7070082F707002DF8070091
:102490000000B0003E0078001000320000277800F5
:1024A0003000200089F707007AF70700C3F707001C
:1024B0001EF807000000B0003E0078000400320063
:1024C0001000B00000277800F0FF2F000200370056
:1024D0000027780000002000020037000027780065
:1024E000F0FF2F00020037000027780000002000D6
:1024F0000200370000277800F0FF2F0002003700AD
:102500000027780000002000801F78003E0078003F
:10251000801F78003E0078003E0078003E00780082
:10252000002778004F007800002778004F007800DF
:102530000000B0003E0078001F0032000027780045
:102540004000200061F7070052F70700FDF7070081
:102550000000B0003E0078000F003200801F7800BD
:102560003E00780000277800000020000027780057
:1025700020002000A5F7070046F7070045F70700F1
:102580004FFA0700002778004F00780000277800F6
:1025900000002000070037003E0078003E00780071
:1025A0003E0078003E0078003E007800002778006A
:1025B000F0FF2F003A0037003E0078003E00780020
:1025C0003E007800801F78003E007800801F780071
:1025D0003E0078002FF707002EF70700002778004D
:1025E00000002000002778002000200099F7070055
:1025F00033FA070027F7070026F707003E007000B0
:102600000000B0003E0078001700320091F707008C
:10261000002778004F007800002778004F007800EE
:10262000002778004000200028F7070000277800E6
:102630004000200025F7070016F7070015F70700F0
:102640001FFA070000277800F0F32F003E0060001B
:1026500000277800600020001CF7070000277800A2
:10266000000020000E003700002778004F0078009F
:10267000002778004F0078003E0078003E00780088
:102680003E0078003E0078003E0078000027780089
:102690003E0068000027780000277800F0FF2F0038
:1026A0000000B0003E00780053FF32000300370006
:1026B000002778003E006800002778000000060030
:1026C000B8010000C44649004E44000022FF070044
:1026D000F0F60700EFF607003E0070000000B000C3
:1026E0003E00780015003200EAF60700E9F6070020
:1026F000F3F90700801F78003E007800002778007B
:102700003E006800002778004F007800002778001E
:10271000F00320003E0060001000B00000277800A9
:1027200030002000CBF70700D3F607006CF7070056
:102730003E0010004100DD0034F7070000000600F5
:1027400040000000415B00000027780000002000EE
:102750004AF907001EF70700000006000E000000FF
:10276000C15D000000277800F0FF2F0043F907004B
:1027700017F70700000006000E000000C13A000035
:10278000002778000002200078FE07006EF907009D
:10279000002778000000200000277800200020009B
:1027A0001AF7070008F9070000277800801F780053
:1027B0003E0078002000B00010007800002778006C
:1027C0007FB897001000780022F707004CFA070046
:1027D0005DF90700002778007FB89700FCF6070036
:1027E000002778004F0078002000B000F8F60700BE
:1027F00000277800F1F6070000277800F00320009A
:102800003E0060001000B000801F78003E0078009D
:10281000002778002000B000E8F6070000277800C5
:10282000F00F20003E0060009AF607001000B00094
:10283000E2F60700002778008000200004F8070077
:10284000002778007FB897001000B10000277800BB
:10285000000C20003E0070003E00400028FA0700F7
:102860003000B000002778004F0078003000B10041
:10287000002778001AF707000000B0003E0078003B
:1028800016003200801F78003E0078000027780094
:102890002000B000C9F6070000277800F00F2000E4
:1028A0003E0060007BF607001000B000C3F6070092
:1028B0000027780080002000E5F707000027780057
:1028C0003000200081F60700BCF6070000277800E2
:1028D000F00F20003E006000DFFF37003E00780070
:1028E0003E00780000277800F0FF2F00E3F8070093
:1028F000B7F6070002F907009DF80700B4F60700D5
:1029000000000600C6000000413B000000277800E0
:10291000600020000027780000002000F8F9070080
:1029200035FA07000027780000002000D3F80700E0
:10293000A7F60700F2F807008DF8070010007800EE
:102940003E0010000000B0003E0078000E00320093
:102950000027780030002000CEF807009CF6070022
:1029600075F8070010007800CAF807002000B000D2
:1029700097F6070076F8070010007800C5F8070002
:102980004000B00092F6070000000600440000007E
:10299000C7495400314D5300212100000027780021
:1029A0004280BF00801F7800004EB30042E0B700B5
:1029B0003E007800BDF8070000277800801F7800EF
:1029C0003E0078002000B00081F607000027780064
:1029D0004F0078007EF60700002778004F0078004F
:1029E00042A0B7003E007800000006003000000062
:1029F000C67370005F7365007100000000277800E7
:102A00004F007800002778004F00780021F607007B
:102A100020F607001FF607001EF6070028F907003A
:102A20003E0070004CF607000000B0003E00780049
:102A300013003200801F78003E00780000277800E5
:102A40000000200000277800600020006FF60700DB
:102A500010F607000FF6070019F9070000277800A5
:102A60004F0078005AF60700002778003E00680003
:102A7000002778002000200064F60700E5FF3700FB
:102A80003E0078003E00780025F807000027780017
:102A9000801F78003E0078006000B0004CF6070010
:102AA000002778007FB897004000B00048F6070084
:102AB00000277800F0FF2700002778007FB89700F4
:102AC0008000B00042F607000027780000002000D8
:102AD000002778007FB897002000B0003CF6070080
:102AE000002778004F00780039F607000000060044
:102AF000B20000004A534500515F4200454749007B
:102B00004E5B0000002778000000200000277800BE
:102B1000804F2100DFF90700002778000000200027
:102B200056F807002AF60700000006001E00000005
:102B3000C7534500515F410044440000E3FE0700D5
:102B4000D4F50700D3F507003E0070000000B00088
:102B50003E007800110032000027780000002000BD
:102B6000AEF9070066F90700002778000000200092
:102B7000BDF9070062F90700002778000000200077
:102B8000BDF507005EF9070000277800000020006F
:102B9000B9F507005AF90700100037003E00780029
:102BA0003E007800002778005000200039F8070028
:102BB00007F60700E0F707001000780035F8070077
:102BC0002000B00002F60700E1F7070010007800CF
:102BD00030F807004000B000FDF5070000000600D7
:102BE0005A000000C8534500515F45004E445D0047
:102BF00000277800000020000027780040F9070037
:102C0000D8FE07000000060014000000C573700025
:102C10005F2E6700002778004F00780000277800BB
:102C20004F0078009BF507009AF50700A4F807000D
:102C300000277800F00F20003E006000801F780021
:102C40003E0078003E00780092F5070091F50700FD
:102C50000027780000002000002778007FB8970048
:102C60001000B000002778003000200079F607003F
:102C700081F507001AF607003E0010004100DD0054
:102C8000E2F50700002778004F0078007AF507008A
:102C9000801F78003E00780077F50700801F7800DD
:102CA0003E0078000000EA005AFB07000000060022
:102CB00068000000C8534500515F4C004953540060
:102CC00097F70700002778004000B0001000780058
:102CD00070F507006000B000100078003E00700042
:102CE0000000B0003E007800B6003200DDF70700BB
:102CF00010007800801F78003E0078001EFC07005E
:102D0000C4FF07001050650072696F006465200001
:102D100064752000544943003A207500002778006C
:102D20001000780000277800801F78003E007800AF
:102D300000277800803E20001CF60700ECFC07000E
:102D400000277800800020001AF80700002778008C
:102D5000C002200017F807008AFC0700B8FC070033
:102D6000B7FC0700B6FC0700DAFC070029FB0700E8
:102D700000277800300720000EF80700FCFA070053
:102D80004000B00000277800801F78003E007800E7
:102D900010007800002778004F0078002000B00075
:102DA000100078003BF507003AF5070044F80700EB
:102DB0003E0070000000B0003E0078007700320056
:102DC0000027780000002000002778002000200065
:102DD0008EF507002FF507002EF5070038F80700DD
:102DE0000027780000002000002778002000200045
:102DF00098F5070027F5070026F5070030F80700CB
:102E0000801F78003E0078003E00780000277800A0
:102E10004F00780000277800002778000008200085
:102E20003E0060000000B0003E0078000900320063
:102E300000277800F00320003E0060000000EA0058
:102E4000F4FA0700DBFA070000277800F0FF2F00F4
:102E500002003700002778003E0068000000B00044
:102E60003E007800DEFF32006AFF0700097065004F
:102E700072696F0064653A002075200000277800B1
:102E80000000200000277800200020005FF50700E8
:102E900000F50700FFF4070009F807000027780095
:102EA0007FB8970000277800803E2000CDF507000E
:102EB0008FFC07000027780080002000BDF7070086
:102EC00000277800C0022000BAF707002DFC070099
:102ED0005BFC07005AFC070059FC07007DFC07005B
:102EE000CCFA07003E007800002778003007200069
:102EF000B0F7070047FF0700092072006574610002
:102F000072643A002075200000277800000020003D
:102F100000277800200020003CF50700DDF40700C2
:102F2000DCF40700E6F70700002778007FB8970079
:102F300000277800803E2000AAF507006CFC0700FF
:102F400000277800800020009AF70700002778000B
:102F5000C002200097F707000AFC070038FC0700B2
:102F600037FC070036FC07005AFC0700A9FA0700E7
:102F70003E00780000277800300720008DF707001A
:102F800000277800000020000027780020002000A3
:102F90001EF5070076FA070082FF37003E00780032
:102FA0003E007800002778004F0078003E0078004F
:102FB000002778004F0078002AF7070004F5070083
:102FC000090037003E00780012FF0700104155004D
:102FD00043554E004520530045515500454E430092
:102FE000452E750062FA0700000006009E010000F1
:102FF00047434F004D5049004C450000D6FC0700A8
:10300000A4F40700A3F407003E0070000000B00025
:103010003E0078000900320097F4070019FA070013
:1030200018FA070000277800000020000027780029
:103030002094200097F80700100037003E00780029
:103040003E007800002778003000200011F70700CC
:10305000DFF40700B8F60700100078000DF707004E
:103060002000B000DAF40700B9F60700100078007D
:1030700008F707004000B000D5F407000000060084
:103080004A000000495B43004F4D5000494C450049
:103090005D000000B0FC07007EF407007DF407002F
:1030A0003E0070000000B0003E00780002003200D8
:1030B00078F80700100037003E0078003E007800E6
:1030C0000027780030002000F2F60700C0F4070067
:1030D00099F6070010007800EEF607002000B00017
:1030E000BBF407009AF6070010007800E9F6070025
:1030F0004000B000B6F40700000006003E000000EB
:10310000C74558004543550054450000801F7800CE
:103110003E007800801F78003E0078000000060026
:1031200012000000C12200000027780040002000AB
:10313000D2F60700F6F5070003F70700002778002E
:10314000F00F20000027780000002000000006009B
:1031500018000000422E2200002778000000200006
:1031600000277800606021004AF80700EEFF0700A2
:10317000000006001200000001280000002778006F
:1031800020002000BDF60700E1F507000000060062
:103190000E000000C22E5300D9F607006EF407009F
:1031A0000000B0003E0078001C00320000277800CC
:1031B00000002000801F78003E0078000027780083
:1031C0001000B000002778007FB897003E00100084
:1031D0003EF40700C6FB0700002778004F00780088
:1031E0001000B00000277800801F78003E007800B3
:1031F00028F40700C7F40700D9F407000000B00066
:103200003E007800EDFF3200002778004F00780084
:103210003E0078003E007800060037007DFE070083
:103220000C5069006C6520007669640065202100FF
:10323000204E4300000006005400000049494D00A4
:103240004D45440049415400450000005EF607002A
:1032500000277800801F78003E0078002000B00032
:1032600010007800002778004F00780010007800E8
:1032700008F4070007F4070011F70700002778009B
:10328000F0F72F003E00600000277800400020008B
:103290001EF4070000277800400020001BF4070000
:1032A0002DF70700000006003800000046444900E2
:1032B000524543005400000043F607000027780001
:1032C000801F78003E0078002000B00010007800D9
:1032D000002778004F00780010007800EDF3070019
:1032E000ECF30700F6F6070000277800F0FB2F004C
:1032F0003E006000002778004000200003F4070033
:10330000002778004000200000F4070012F70700B3
:103310000000060036000000C5414C004C4F540030
:10332000002778000000B0003E0078000500320061
:103330000027780000002000CBF707001000B10044
:10334000F7FF37003E007800000006001C00000078
:10335000C44C4F00414400004EF6070010007800B6
:103360000000B0003E007800020032003E0078000D
:10337000E9013700F0F5070010007800801F7800A1
:103380003E007800F2F5070010007800801F7800FA
:103390003E00780027F6070010007800801F7800B4
:1033A0003E00780029F6070010007800801F7800A2
:1033B0003E007800E0F5070005F4070000277800DC
:1033C00000002000E2F5070001F407002BF60700DB
:1033D000100078000027780041F407000000B000DA
:1033E0003E007800B6003200002778002000200060
:1033F00054F407000000B0003E007800A100320045
:10340000002778002002200058FB070024FA07005C
:103410000027780030002000ACF307000027780078
:10342000F00F200035F407009AF307002CF4070092
:103430003E0060000000B0003E0078002C0032002A
:10344000801F78003E007800801F78003E007800E2
:1034500089F30700C0F307000000B0003E007800C9
:1034600017003200002778000027780000102000A5
:1034700022F407000000B0003E007800080032008F
:10348000002778007FB89700CCF30700002778006A
:1034900080002000EEF407003E00400007003700E7
:1034A000002778007FB89700C4F3070072F3070085
:1034B00013F7070000277800000020000300370002
:1034C000002778007FB89700BCF307006AF3070075
:1034D0001000B000002778004F0078001000B00006
:1034E000002778004F0078001000B100C8FF3700B7
:1034F0003E007800B1F3070000277800002778002D
:103500002002200009F407000000B0003E0078000F
:103510002A0032003E007800801F78003E007800CC
:103520008DF307000000B0003E0078000400320078
:1035300000277800000020004FF30700F0F6070096
:1035400054F3070053F307005DF6070000277800E7
:1035500000F02F003E006000002778004F00780048
:103560003E004000002778004000200057F307008D
:10357000002778004000200054F3070076F607008B
:10358000BEF507001000780000277800300020000A
:10359000E6F307000000B0003E00780002003200B1
:1035A0003E0078003E0078000027780040002000B0
:1035B000B2F50700DEF4070031003700A3F507007D
:1035C000100078000000B0003E00780003003200D8
:1035D0003E00780000277800D00020002DF307007F
:1035E00000277800F00F2000C4F307000000B000AF
:1035F0003E00780021003200801F78003E007800F5
:103600001DF3070054F307000000B0003E007800EF
:1036100015003200002778000027780000102000F5
:10362000B6F307000000B0003E007800070032004B
:10363000002778004F0078000027780080002000E5
:1036400083F407003E0040000600370000277800A2
:103650004F00780008F30700A9F60700002778005C
:103660000000200002003700002778004F0078009B
:1036700001F307001000B000010037003E007800A1
:103680000E0037000027780000022000B7FA07007C
:10369000100078000027780010902200A3F30700A4
:1036A0000000B0003E0078000400320000277800DF
:1036B0002000200071F507009DF40700EB003700A3
:1036C0003E00780024FB0700F2F20700F1F2070049
:1036D0003E0070000000B0003E0078005F00320045
:1036E00066F50700100078000000B0003E0078008A
:1036F00024003200E7F20700E6F20700F0F50700C9
:10370000DDF207003E007800002778000008200066
:103710003E0060000000B0003E0078000200320071
:10372000DCF6070016003700DAF20700D9F20700CE
:10373000E3F50700801F78003E007800002778003E
:103740003E006800002778004F00780000277800CE
:10375000F00320003E0060001000B0000027780059
:1037600030002000BBF30700C3F207005CF3070042
:103770003E0010004100DD0024F3070063FE070057
:1037800035003700C3F20700C2F20700CCF507008E
:10379000B9F207003E00780000277800000C2000F6
:1037A0003E00600000277800000420005FF307005F
:1037B0000000B0003E007800110032003E007800AA
:1037C0003E007800002778002000200031F5070037
:1037D000FFF20700D8F40700100078002DF507006D
:1037E0002000B000FAF20700D9F4070010007800BA
:1037F00028F507004000B000F5F20700160037007A
:10380000A4F20700A3F20700ADF50700801F7800BF
:103810003E007800002778003E006800002778000E
:103820004F00780000277800F00320003E00600081
:103830001000B000002778003000200085F307005A
:103840008DF2070026F307003E0010004100DD0066
:10385000EEF207002DFE0700840037003E007800DE
:103860008EF4070000277800D4F207000000B000B3
:103870003E0078007B00320086F2070085F20700E8
:103880004EF9070089F207003E00780087F2070032
:103890003E00780000277800C8F207000027780073
:1038A000100220001BF307000000B0003E0078006B
:1038B000080032003E007800F0F4070010007800A5
:1038C0000000B0003E00780001003200EDF7070074
:1038D0006300370000277800B8F20700002778005F
:1038E00000277800B002200010F3070062F2070002
:1038F00000277800D00220000CF307003E00700083
:1039000064F207001000B000ACF207000027780056
:1039100010022000FFF207003E0060000000B0002F
:103920003E0078003E0032005AF207000000B0006E
:103930003E00780037003200A0F20700CFF4070005
:10394000100078000000B0003E0078002700320030
:10395000801F78003E00780000277800002778005C
:1039600000402000E5F207000000B0003E007800B3
:103970000E0032000027780040002000B4F307005A
:10398000002778004F00780000277800D002200040
:10399000E6F2070000277800100020003E006000DB
:1039A000000BB00034F207000E003700B5F7070037
:1039B0000027780000042000002778004F007800DE
:1039C00000277800D0022000D8F2070000277800F6
:1039D000000320003E0060003E0010000027780039
:1039E000E0032000C6F50700090037000027780033
:1039F000B0022000CDF207000000B0003E007800C9
:103A0000020032003E004000010037003E0010007E
:103A1000020037003E0078003E00780010003700BA
:103A20003E0078003E00780000277800100020005B
:103A300098F4070066F207003FF4070010007800D2
:103A400094F407002000B00061F2070040F4070082
:103A5000100078008FF407004000B0005CF207000F
:103A6000020037003E0078003E00780077F407003F
:103A70001000780087F40700100078003E00700006
:103A80000000B0003E00780050FE32009CF40700B9
:103A90004F80DE000000B0003E0078000E003200D3
:103AA00000277800400020007AF4070048F2070061
:103AB00021F407001000780076F407002000B00021
:103AC00043F2070022F407001000780071F40700A9
:103AD0004000B0003EF20700002778004F00780059
:103AE0005AF407003AF20700002778004F007800E8
:103AF00050F4070036F20700002778004F007800E6
:103B000013F4070032F20700002778004F00780016
:103B100009F407002EF2070000000600E803000089
:103B2000C64352004541540045000000BBF5070064
:103B300054F7070084F407001DF4070000277800FD
:103B4000801F78003E00780021F2070000277800EF
:103B50004F0078002000B0001DF207000027780019
:103B60004000200000277800F0FF2F0064F50700D8
:103B7000002778000000200000277800F0072000D0
:103B80005FF507009CF50700000006003800000004
:103B9000C87370005F646F0065733E0004F4070033
:103BA00000277800801F78003E0078002000B000D9
:103BB00010007800002778004F007800100078008F
:103BC0000027780000002000002778004F007800D0
:103BD0000027780040002000BCF107000027780093
:103BE00040002000B9F10700002778000000200005
:103BF000002778002000200004F20700D6F4070018
:103C00000027780040002000002778004F0078004F
:103C10000027780040002000BCF107000027780052
:103C200040002000B9F10700CBF4070072F507004F
:103C3000002778000000200010F40700E4F10700DE
:103C4000000006009400000045444F0045533E002C
:103C500000277800000020000027780080DC210089
:103C60008CF507000000060012000000C856410055
:103C700052494100424C4500C1FA0700ABFF070022
:103C800079F50700C5FF07000000060012000000DC
:103C9000C8434F004E535400414E5400B8FA070039
:103CA000F8F6070000277800600020000027780061
:103CB0000000200012F507004FF5070000277800EC
:103CC00000002000EDF30700C1F10700000006002E
:103CD00022000000C653540052494E004700000025
:103CE000A7FA070064F10700E6F60700E5F607000B
:103CF00000277800600020000027780000002000E6
:103D0000FFF407003CF507000027780000002000C2
:103D1000DAF30700AEF107000000060026000000FD
:103D2000C5564C0049535400A7F3070000277800FC
:103D3000801F78003E0078002000B000100078005E
:103D4000002778004F0078001000780051F107003C
:103D500050F107004FF107004EF1070058F407003B
:103D6000801F78003E0078003E0078000027780031
:103D70004F00780000277800F00320003E0060002C
:103D80000000EA0023F707000AF7070041F10700E7
:103D900040F107000027780000002000002778008D
:103DA00020002000ABF1070045F4070039F10700BF
:103DB00038F107003E0070000000B0003E007800BF
:103DC00004003200A3F10700002778000000200063
:103DD000040037003E0078003E007800002778009D
:103DE000F0FF2F000000B0003E007800D7FF320047
:103DF0003E0078003E0078000000060070000000E1
:103E0000C34B450059000000B0F3070000277800BD
:103E10001000B00069F107000140FE001DF107002D
:103E200066F107001BF107003E0010000000B00023
:103E30003E007800F8FF320016F107003E00400017
:103E40002000B0005DF10700801F78003E00780080
:103E50001000B0000027780058F107001000B000F3
:103E600000277800F00720003E00600002F1070004
:103E70005CF10700002778004F0078000000060082
:103E800042000000C5494E004B4559008FF3070022
:103E90000027780049F10700002778000027780004
:103EA0003000200009F107001000B0004DF10700BC
:103EB0001000B10000277800F00720003E006000ED
:103EC0003E0040002000B0003CF10700000006006A
:103ED00028000000C84B450059424F0041524400A1
:103EE0007AF307001000B000002778001000B1003E
:103EF00032F10700E7F0070030F107003E00100044
:103F00000000B0003E007800060032000027780074
:103F10002AF107003E0040001000B00027F1070022
:103F200002003700002778003E006800000006000D
:103F300030000000C64558005045430054000000C2
:103F400000277800F00F20003E0060000027780076
:103F5000000020000027780030002000DBF0070080
:103F600020F10700CBF007001000B000C9F00700F7
:103F7000002778000002200076F20700A2FF070069
:103F80000027780000277800F00120006DF107007D
:103F9000C0F0070000277800F00720005DF107005F
:103FA0003E006000BBF00700002778009000200072
:103FB0005EF107003E0070000027780040002000FE
:103FC000C2F00700FDF00700002778004000200045
:103FD000BEF007004FF107003E0060000000B00097
:103FE0003E00780047003200002778000027780064
:103FF000900020004DF107000000B0003E00780066
:10400000180032003E0078000027780000022000EF
:104010000027780080002000002778004000200062
:10402000AAF00700E5F0070000277800801F78005D
:104030003E00780000277800700020003E006000FD
:104040003E00100000277800300020009FF007009D
:10405000002778004F0078003E001000D1F10700E3
:10406000020037000027780010002000801F780031
:104070003E00780000277800801F78003E0078001E
:10408000002778004BF3070000277800300020005D
:104090008EF00700C9F007001000B000002778007C
:1040A0004000200089F00700CEF0070000277800CC
:1040B0003000200085F0070000277800BFF00700DF
:1040C0003E004000C7F00700002778004F0078004E
:1040D000002778004F0078001000B100002778001A
:1040E000F8F007000000B0003E007800DFFF32006B
:1040F0003E0078003E007800002778000000200095
:104100004F0037000027780000277800F0072000D4
:1041100006F107005FF0070000277800800020000C
:1041200002F107003E0070005AF0070000277800F7
:10413000C0012000FDF007003E007000002778005D
:104140004000200061F007009CF00700E4F0070049
:104150003E0060000000B0003E0078001400320015
:104160003E0078004BF0070094F00700002778002D
:10417000100020003E0010000027780030002000D2
:1041800052F0070097F00700002778008000200019
:1041900008F3070007F607000027780080002000DA
:1041A00004F30700002778000000200024003700F7
:1041B000002778000027780030002000DBF007009F
:1041C00034F0070000277800D0002000D7F0070067
:1041D0003E0070002FF00700BAF007003E007000AC
:1041E0000000B0003E0078000B003200002778008D
:1041F0003000200035F00700002778006FF007003E
:104200001000B0003E00400076F007000027780064
:10421000F0FF2F000A00370000277800A0002000E0
:10422000C2F00700CEF007000000B0003E007800AA
:1042300001003200D8F507000027780000002000B8
:104240000000B0003E0078004CFF32003E007800D5
:104250003E0078000000060094010000C4515500A3
:10426000495400000F802000002778000000200043
:104270000027780081F2070055F0070085F207005B
:1042800053F007007DF207001000780032F00700BD
:104290000000B0003E0078001500320000277800D2
:1042A0004F80DE000000B0003E00780004003200C5
:1042B0003E00780000277800A00320000B003700A4
:1042C00000277800200020009EF007000000B000CA
:1042D0003E00780003003200002778002002200012
:1042E000020037000027780080022000020037001B
:1042F00000277800E0032000AEF20700E0F107009D
:1043000000277800F8F10700100078000000B000E6
:104310003E0078000300320000277800F0052000FE
:104320000200370000277800E004200004FF0700A7
:104330008FF507000027780030002000D5EF070038
:10434000002778001DF007003E0040001000B0007C
:1043500024F007000027780000002000CDEF0700C0
:1043600020F007001000B000DFF107001000780017
:104370000000B0003E0078000800320000277800FE
:10438000300120008BF20700F3FB070000277800C4
:104390001001200087F2070001003700EEFB070044
:1043A0003CF20700100078000000B0003E007800EA
:1043B000B50032000E902000CBF10700100078000D
:1043C0000000B0003E00780009003200C4FE070083
:1043D0000000B0003E007800020032008AFE0700B4
:1043E0003E0078000027780000002000020037001F
:1043F00000277800F0FF2F000000B0003E0078009A
:10440000EDFF32001DF20700100078000027780051
:10441000F0FF2F0045F007000000B0003E007800DC
:1044200020003200E8F1070000277800801F7800A4
:104430003E0078002000B0001000780000277800CF
:104440007FB897001000780092EF070091EF070007
:1044500090EF07008FEF0700002778000000200092
:104460000027780020002000FAEF070094F20700F0
:10447000F8EF0700002778007FB89700D4EF070017
:10448000002778004F0078002000B000D0EF070030
:104490003BF207000027780000002000F7F107003A
:1044A000CBEF0700DBF90700052A2A002A2A2000A3
:1044B0007AF10700FAF5070056F507003DF5070009
:1044C000F4F107001000780000277800002778003A
:1044D0001000200015F007000000B0003E0078003A
:1044E0000A003200CBF90700183A2000496E730029
:1044F00074727500637469006F6E2000494E43004A
:104500004F4E4E005545200021747800002778005A
:10451000002778002000200004F007000000B00011
:104520003E0078000A003200BAF90700193A20006C
:10453000496E730074727500637469006F6E2000B9
:10454000494D4D0045444900415445002021780023
:10455000002778000027780030002000F3EF0700E4
:104560000000B0003E0078000B003200A9F90700FF
:104570001B3A200050524F00424C45004D45200050
:1045800050696C00652064006520520045544F005E
:1045900055522000210D5400002778000027780094
:1045A00040002000E1EF07000000B0003E0078006E
:1045B0000B00320097F907001D3A200050524F00BF
:1045C000424C45004D45200050696C006520640058
:1045D00065732000444F4E004E4545005320210096
:1045E000002778000027780050002000CFEF070058
:1045F0000000B0003E0078000E00320085F9070090
:1046000024494D00504F5300534942004C4520006F
:10461000642769006E73650072657200206365002F
:104620007474650020534500515545004E434500C4
:10463000215F6300002778000027780050002000E9
:10464000C0EF07000000B0003E0078000800320014
:1046500070F907000C3A20004552520045555200AF
:10466000206E6F0020276900A1F6070001003700C7
:104670003E007800C8F40700BDF40700002778006A
:10468000F0FF2F000F0037007CF1070010007800CA
:104690008CEF07000000B0003E00780007003200F9
:1046A00000277800F0042000C2F1070000277800FE
:1046B000B0042000BFF10700ADF407000027780028
:1046C000000020000000B0003E007800EDFE320047
:1046D00000277800000020000000B0003E007800B5
:1046E000E0FE32000000060048020000C541420022
:1046F0004F5254000E902000BFF2070000277800B0
:1047000000002000002778000BF1070030EF0700C1
:104710000FF107002EEF070095F407003DF90700A1
:10472000262A2A002A2A2000494E540045525200C7
:1047300055505400494F4E00204C6F00676963008C
:1047400069656C006C652000284142004F5254009E
:104750002920210086F407008FF40700C1FE07001E
:104760000000060000277800600320000027780082
:10477000801F78003E007800100078000027780045
:104780004F0078000027780010002000DDF00700BF
:104790005FF007000EEF07000040060000277800DA
:1047A0006003200000277800801F78003E0078001A
:1047B00010007800002778004F007800002778006C
:1047C0001000200006F1070051F0070000277800D4
:1047D0004008200000277800801F78003E00780005
:1047E000100078000027780070FF2F003E00600066
:1047F000002778004F007800F5EE0700BAF00700B8
:10480000100078000000B0003E0078002C0032005C
:10481000B5F0070000277800801F78003E00780080
:10482000100078001000B100002778000027780001
:104830004F007800E6EE070022EF07000000B0000E
:104840003E0078001E00320020F1070000277800AB
:10485000DAEE07001000B00000277800F007200013
:104860003E0060008BEE07001000B000D3EE0700A2
:1048700088EE07002DEF07000000B0003E00780032
:10488000030032003E0078003E0078000C00370044
:1048900000277800D000200000277800300020009A
:1048A0008AEE070000277800C4EE07003E004000B3
:1048B0002000B000CBEE07006FEE0700C9EE070046
:1048C000FAF0070000277800801F78003E0078008B
:1048D00010007800002778004F0078002000B0001A
:1048E000100078006BEE07006AEE07003E007000D3
:1048F0000000B0003E0078000200320003FA07001A
:10490000020037003E0078003E00780084F0070087
:10491000002778008000B000100078001000B00080
:104920004F80DE000000B0003E007800370032000B
:10493000BAF0070000277800801F78003E0078005A
:1049400010007800002778004F0078002000B000A9
:10495000100078004FEE07004EEE07003E0070009A
:104960000000B0003E0078002600320000277800EA
:104970000000200000277800A8F00700002778003A
:10498000801F78003E00780091EE07000027780035
:104990004F0078002000B0008DEE070066F00700A1
:1049A000100078000000B0003E00780012003200D5
:1049B00000277800F00720003E0060000027780004
:1049C0004F0078000027780000F82F003E006000BC
:1049D0003E004000002778004F0078003E0078003D
:1049E00025EE0700801F78003E007800801F7800C9
:1049F0003E007800020037003E0078003E0078005C
:104A0000020037003E0078003E0078000027780062
:104A1000100078000000B0003E00780094003200E2
:104A2000002778002000B000100078001000B100CE
:104A3000002778004F80DE000000B0003E007800C4
:104A40008800320013EE0700100078003E0040009E
:104A500010EE07002000B0005DEE07000027780090
:104A6000000020000BEE07004000B0000027780097
:104A7000801F78003E007800100078000027780042
:104A80004F0078002000B0001000780001EE070011
:104A900000EE07000AF107003E0070002EEE07004E
:104AA0000000B0003E0078006A003200801F7800ED
:104AB0003E007800801F78003E007800801F78005C
:104AC0003E0078001000B000002778004F0078000A
:104AD000002778004F007800002778007FB8970003
:104AE000100078001000B100002778004F80DE0031
:104AF0000000B0003E0078004D0032000027780032
:104B000050002000F1ED07008000B0001000780098
:104B10000027780050002000ECED070089EE070028
:104B20000000B0003E0078003D003200801F780099
:104B30003E007800D7ED0700D6ED0700002778008B
:104B40000000200000277800400020002FEE070022
:104B5000DBF00700002778004F0078003E0040009F
:104B6000002778004F00780019EE07003E0078001B
:104B70000027780040002000D4ED07008000B0003E
:104B800000277800801F78003E0078001000780031
:104B90000027780040002000CCED070000277800B7
:104BA0004F0078000AEE0700002778003000200050
:104BB000C6ED07000027780030002000C3ED070095
:104BC0000027780000002000002778002000200047
:104BD0000EEE0700BAF00700002778004280BF0001
:104BE000801F78005FF89700004EB20042E0B700E7
:104BF0003E00780045F90700002778004F00780054
:104C000042A0B7003E007800002778005000200046
:104C1000AEED07008000B000EDED070003003700A7
:104C2000002778004F007800E9ED07000300370007
:104C3000002778004F007800E5ED07000027780096
:104C4000000020000027780080002000EFED070022
:104C50008EFF37003E0078003E0078003E0078006E
:104C6000030037008BED07002000B000D8ED0700EF
:104C70003E007800D6ED07000040060000277800CF
:104C80006003200000277800801F78003E00780035
:104C900010007800002778004F0078000027780087
:104CA00020212000C5ED07000027780040082000E3
:104CB00000277800801F78003E0078001000780000
:104CC00000277800F0DF2F003E006000002778000A
:104CD0004F007800BEED07007DEF07000027780049
:104CE000801F78003E0078002000B000100078009F
:104CF000002778004F0078001000780065ED07006D
:104D000064ED07003E0070000000B0003E00780037
:104D100002003200FDF80700460037003E00780030
:104D20003E007800002778001000B1000000B000BD
:104D30003E0078003200320000277800002778001B
:104D400030012000F9ED070052ED07000027780040
:104D500010012000F5ED07003E0070000000B000DB
:104D60003E00780007003200002778003001200064
:104D7000EEED0700D5EF07002008B00099ED070021
:104D80001E003700D1EF0700002778008BED0700E9
:104D90001000B00000277800F00720003E006000FF
:104DA0003CED07001000B00084ED070039ED07006E
:104DB000DEED07000000B0003E0078000400320085
:104DC0003E0078003E0078003E0078000B0037007F
:104DD00036ED070000277800300020003BED07008B
:104DE0000027780075ED07003E0040002000B0006D
:104DF0007CED070020ED07007AED07000D0037007D
:104E0000002778003E006800002778006037220005
:104E100082EF070000277800801F78003E007800AE
:104E20006BED0700002778004F0078002000B000ED
:104E300067ED070066ED070000400600AA030000CA
:104E4000D15449004D455200315F55004152540044
:104E5000315F49004E495400002778003099230003
:104E6000002778002010200059ED07000027780067
:104E700000002800002778004010200054ED0700B3
:104E800000277800700020000027780040212000D3
:104E90004FED070000277800000020008BEF07008F
:104EA0004BED07000027780000402800002778001D
:104EB000C020200046ED07000027780000402000B9
:104EC00000277800E020200041ED0700002778004F
:104ED0008020200000277800C00820003CED07005B
:104EE000002778000000200006EF070038ED0700DB
:104EF000000006005C000000C55445004D504F0006
:104F000037EF0700100078000140FE00E1EC0700D9
:104F100033EF0700100078000027780030002000F1
:104F2000EAEC07003E00100074ED07000000B0003E
:104F30003E007800F4FF32003E0078003E0078002A
:104F40000000060028000000C5464F0052544800EB
:104F500030F70700CD0D45006E747200657A2000B1
:104F600064616E0073206C0065206D006F6E6400DC
:104F700065206400752046004F525400480D0D0016
:104F800020202000202043006F70790072696700A4
:104F9000687420006A7062002E666F007274680088
:104FA0000D0D4E006F79610075205300455155007D
:104FB000454E43004555520020706F007572200029
:104FC000647350004943330030460D00205665009D
:104FD000727369006F6E2000312E30003020200087
:104FE0006475200032322F0030352F00323031000E
:104FF000360D20002068740074703A002F2F6A006C
:1050000070622E00666F720074682E006672650012
:10501000652E6600722F0D0020206A0070625F000E
:10502000666F720074684000796168006F6F670096
:10503000726F750070732E00636F6D000D0D200090
:1050400051756500206C650020464F0052544800A1
:1050500020736F006974200061766500632054003E
:105060004F4921000D0D6E00000006009400000065
:10507000C6464F005247450054000000B6F40700F2
:1050800084EC070083EC07003E0070000000B000D5
:105090003E0078001D0032007EEC07007DEC07002A
:1050A0000027780000002000002778002000200062
:1050B000E8EC070077EC070076EC070030EF07001C
:1050C0007FEF0700E3EC0700BFEE07000027780042
:1050D000801F78003E007800BDEC070000277800B4
:1050E0004F0078002000B000B9EC070000277800DE
:1050F000F00F200000277800F0FF2F0012EF0700CC
:1051000095EF07003CF00700020037003E007800F2
:105110003E0078000000060056000000CE54450016
:105120004C4543004841520047454D00454E540010
:105130000027780080BB20006BEE0700A4EC07007E
:105140000000060016000000C94445004D41520011
:105150005241470045000000A08A200020A0B7006F
:105160000F8020000E9020000E0078007F020900C2
:105170000018EB000027780010002000DAEE07008E
:1051800093EC07000027780080B5200029F0070085
:1051900000277800F0FF270061EE07008000B000D4
:1051A0008BEC07002CFF0700FBF2070000277800BC
:1051B00000002000002778000010200040EF0700CA
:1051C00034EC070033EC07000027780000002000D3
:1051D00000277800200020008CEC07002DEC070051
:1051E0002CEC070036EF0700801F78003E007800A7
:1051F00000277800F00F2000CCEC07000027780093
:105200004F00780000277800F0FF2F00C7EC070060
:105210003E0060000000B0003E007800EAFF32006F
:105220001CEC07001BEC0700D5EE070019EC07008B
:10523000002778005000200024EC0700BBEC07009A
:1052400014EC070000277800500020001FEC070036
:10525000B6EC07003E0060000000B0003E007800A1
:10526000050032003E0078003E00780000277800FC
:10527000F0FF2F006900370006EC070005EC07007F
:105280000027780000002000002778002000200080
:1052900070EC07000AEF0700FEEB07000000B0000B
:1052A0003E0078000A0032003E0078003E007800A0
:1052B0000027780000002000002778002000200050
:1052C00064EC07000027780000002000530037003E
:1052D000801F78003E007800801F78003E00780034
:1052E000ECEB0700EBEB0700002778004F0078009D
:1052F000002778004F00780056EC0700E5EB070028
:105300004F80DE000000B0003E0078000C0032004C
:105310003E0078003E007800002778000000200062
:1053200000277800200020004AEC070000277800C2
:105330000000200000277800F0FF2F003400370025
:10534000D4EB07000027780070002000DFEB070097
:1053500076EC0700CFEB07000027780070002000F4
:10536000DAEB070071EC07003E0060000000B000BF
:105370003E0078000A0032003E0078003E007800CF
:10538000CAEB07003E007800C8EB07003E0078003B
:1053900000277800F0FF2F00002778001C0037005E
:1053A000BCEB0700BBEB07000027780000002000E3
:1053B000002778002000200026EC0700C0EE070040
:1053C000B4EB07000000B0003E0078000E00320091
:1053D0003E0078003E0078003E0078003E007800F5
:1053E000002778000000200000277800200020001F
:1053F00018EC070000277800000020000027780044
:10540000F0FF2F0002003700002778000000200086
:105410000000B0003E007800B7FF32000000B0008E
:105420003E00780081FF32009AEB070099EB0700FD
:10543000E5ED070000277800801F78003E00780027
:10544000E3EB0700002778004F0078002000B00051
:10545000DFEB07008FEB07008EEB070098EE0700ED
:10546000801F78003E00780000277800100420009C
:105470002EEC0700002778004F0078000027780006
:1054800050CC240029EC07003E0060000000B00072
:105490003E00780020003200002778000000200045
:1054A0000027780020002000D8EB070079EB0700E8
:1054B00078EB070082EE0700801F78003E0078003E
:1054C000002778005004200018EC0700002778001F
:1054D0004F00780000277800E034240013EC070028
:1054E0003E0060000000B0003E007800070032007F
:1054F000002778000000200000277800200020000E
:10550000C2EB070001F70700020037003E007800F9
:105510003E007800020037003E0078003E00780030
:1055200015F207008AFE07001BF107004DFB07007C
:1055300000000600FFFFFF00FFFFFF00FFFFFF006E
:00000001FF
